S02200006963632D612D312D626F6F746C6F616465722D636F6D62696E65642E733337F1
S31500000000002000200D0500005905000059050000DC
S315000000105905000059050000590500005905000062
S315000000205905000059050000740500005905000037
S315000000305905000059050000590500005905000042
S3150000004010B5054C237833B9044B13B10448AFF30C
S3150000005000800123237010BD100100200000000065
S315000000608805000008B5034B1BB103490348AFF3ED
S31500000070008008BD00000000140100208805000073
S315000000800E4B0F4A9A60D3F8882042F47002C3F8E8
S3150000009088200C4B5A6D42F400525A651A6C22F0B5
S315000000A003021A64084A136823F00103136052F826
S315000000B0143C23F0805342F8143C704700ED00E0F6
S315000000C00000000000300E4074300E400F4A70B53C
S315000000D0002308258B4201D1002070BD50F8234033
S315000000E094610B4CD5600133D669F60705D514B972
S315000000F06FF00200F1E7013CF6E7002CF8D0D46976
S31500000100A407E7D56FF00100E7E700BF00000E4047
S3150000011080969800094A0A4BD969C90705D512B9CC
S315000001206FF002007047013AF6E7002AF8D0012284
S315000001301861DA60D86940F38000704780969800AD
S3150000014000000E4009B1FFF7C1BF08467047000026
S31500000150234B2DE9F0470F4641F671311E6C1964A9
S31500000160996841F001018146B6B299604FEA92085A
S31500000170BA46002545450ED30020D9F800203B6835
S315000001809A420ED04846FFF7C5FF50B901213846BE
S31500000190FFF79CFF05E009EB85042046FFF7BAFF51
S315000001A048B10F4B9A6822F001029A600EB1002204
S315000001B01A64BDE8F087C4F30A04C4F50064A40811
S315000001C0A8EB05039C4228BF1C4621465046FFF774
S315000001D0B9FF0028D1D125440AEB840ACAE700BF3B
S315000001E000000E401E4B41F671311A6C10B51964B1
S315000001F0996841F00101996001211861D960D969B6
S315000002004C0792B209D5996821F0010199600AB1AB
S3150000021000221A644FF0FF301FE00221114CD96012
S315000002201946D869C00700D56CB9C8698B6810F043
S31500000230020023F001038B6007D00AB100230B6490
S315000002406FF0010009E0013CEBE724B902B10C6450
S315000002506FF0020001E00AB1086410BD1046FCE729
S3150000026000000E4080969800FFF772BF08B5074B56
S315000002701A68074B1A6000F06FF80028FBD040F2AE
S31500000280022000F09FF8002008BD00BF04010020F6
S315000002900001002010B5104C0023A36000F0B2F856
S315000002A00E4B5B68B3F5803F09D040F209239842B4
S315000002B002D0B0F5007F02D100F012F858B94FF421
S315000002C00063A3601846016881F3088881F30988F2
S315000002D040688746FEE710BD00ED00E000500E4086
S315000002E0F8B528231A681069D568836AAB4201D22B
S315000002F00020F8BD05F560529A42F9D95B1BC61875
S31500000300C758134B9F42F3D14FF0FF32F16800F00C
S31500000310E1F8104B98420446EAD140F628031B68E0
S31500000320A3F50062B2F5605F10D21A68BA420DD129
S31500000330B1689A68914209D84FF0FF32D9682846C9
S3150000034000F0C8F8001B18BF0120D2E70120D0E753
S3150000035007B0CD5EE320BBDEF8B528231B68D3E9E2
S315000003600347BB6A1B1BFD182646EA68A318B3425F
S315000003701BD83946204600F078F8A8B140F6280385
S315000003801B68A3F50062B2F5605F14D219680B4AC8
S31500000390914210D1D9684FF0FF32204600F09AF80A
S315000003A0074BC31A58425841F8BD304600F056F87C
S315000003B006F50066D9E70020F6E700BF07B0CD5E78
S315000003C0E320BBDE4FF000534FF20F025A800A4A79
S315000003D01880136823F4E06343F400731360BFF3DB
S315000003E04F8F0649064BCA6802F4E0621343CB609E
S315000003F0BFF34F8F00BFFDE700500E4000ED00E059
S315000004000400FA054FF000534FF20F015A888A4252
S3150000041001D1188870473AB91B88012B40F2022097
S3150000042018BF4FF4007070474FF40070704707B55F
S3150000043003469B0753BF6FEA01414FF6FF7343EA3A
S3150000044001416FEA11410422019120F003000DEBF6
S315000004500201FFF709FF03B05DF804FB08B5FFF7DB
S31500000460C1FEB0FA80F0400908BDF8B540EA0203C3
S315000004701446DA0705460E4601D50020F8BD0CB92C
S315000004800120FBE7830721D50988FFF7D0FF002865
S31500000490F3D1023C032C05F1020506F102060BD945
S315000004A024F003073A4631462846FFF7DDFE0028CA
S315000004B0E3D13E443D44E41B002CE1D0318828467C
S315000004C0FFF7B5FFB0FA80F04009D7E7032CE7D86D
S315000004D0F4E7000010B50B4CD4F8B03043F020031D
S315000004E0C4F8B030084B01241C6001449A605C607B
S315000004F01A46884201D1D86910BD10F8014B9461A3
S31500000500F7E700BF00400E4000C001400B4880479F
S315000005100B4880470B490C4A0C4B9A42BEBF51F818
S31500000520040B42F8040BF8E709490A4A00209142F5
S31500000530BCBF41F8040BFAE7FFF798FE8100000004
S31500000540950200008C05000000010020100100202B
S31500000550100100202C010020FEE700BFF8B500BF07
S31500000560F8BC08BC9E467047F8B500BFF8BC08BC8E
S315000005709E467047AD1007B00100000000030A0157
S31500000580000800000080000000000000C0EA210111
S31100000590C0EA21016500000041000000E7
S31500000800007C0020D1080000CD080000AD090000E2
S31500000810CD080000CD080000CD080000CD0800007E
S31500000820CD080000CD08000024370000CD080000E8
S31500000830CD08000058370000CD080000CD080000A4
S3150000084010B5054C237833B9044B13B10448AFF304
S3150000085000800123237010BD180100200000000055
S31500000860F039000008B5034B1BB103490348AFF349
S31500000870008008BD000000001C010020F0390000C7
S315000008800E4B0F4A9A60D3F8882042F47002C3F8E0
S3150000089088200C4B5A6D42F400525A651A6C22F0AD
S315000008A003021A64084A136823F00103136052F81E
S315000008B0143C23F0805342F8143C704700ED00E0EE
S315000008C00008000000300E4074300E40FEE70000C5
S315000008D008B5FFF7D5FF00F0D9F80A4A0A4B0B49CD
S315000008E08B4206D30A4B0B4A0021934206D300F0F3
S315000008F061F852F8040F43F8040BF1E743F8041BC0
S31500000900F3E700BFF03900000001002018010020C5
S3150000091018010020EC0300200020704700207047DB
S3150000092030B51C4B87B001AA03F110051868596849
S31500000930144603C40833AB422246F7D11B78164A45
S315000009402370D2F8943003F00703022B1ED01369EC
S31500000950C3F30443102B1BD806A90B440F4913F805
S31500000960140C0F4B43438B4206D111690122C1F38C
S3150000097041618A40B3FBF2F3074AD2F80001C0F3A3
S3150000098004200130B3FBF0F007B030BD054BF3E7B0
S31500000990054BF1E71037000000400E4000093D000E
S315000009A040420F0000F04902C0EA21014FF40170F5
S315000009B002F008B92F4B13B501225A642E4BDC6C9A
S315000009C001A8240E00F078FF8E2C1CD82B49D1F8F4
S315000009D0B00040F00403C1F8B030294B4FF050127C
S315000009E01A601A631A66C3F89020C3F8C020C3F8C9
S315000009F0F020C1F8B000214AD36A23F07F0343F008
S31500000A002003D36201E08F2CF5D99DF80530012B28
S31500000A1001BF1C4A136843F0040313601A4B0022FB
S31500000A201A60FFF779FF02F0C6F801F043FD01F006
S31500000A3043FD18B14FF4017002F0C4F801F06AFDED
S31500000A40044601F0F7FE1CB140F203739C4203D149
S31500000A5040F2012002F0B6F8A4F20574012C94BF0E
S31500000A6040F203204FF4017002F0ACF8002002B00F
S31500000A7010BD00BF00000E40B081E00F00400E40E8
S31500000A8000A0004064310E40B40AC64308B51C4BB2
S31500000A905B685B050FD400F07DFF80F00100C0B2FB
S31500000AA044F204031B68013314D14FF40270BDE80D
S31500000AB0084002F079B802F0A5F8A0F2022080B250
S31500000AC00728E8D8012303FA00F010F0C90FE2D096
S31500000AD00020E5E790B14FF4804001F0D9FF0028EF
S31500000AE0E3D0084A4FF4804393601846016881F3C7
S31500000AF0088881F3098840688746FEE708BD00BF7D
S31500000B0000500E4000ED00E00020704749BA89B25F
S31500000B104840C0F30311414008B280EA013000B2F8
S31500000B20C3B280EA431080B2704738B50446451810
S31500000B301046AC4200D138BD014614F8010BFFF750
S31500000B40E5FFF6E710B50B4CD4F8B03043F02003C0
S31500000B50C4F8B030084B01241C6001449A605C6004
S31500000B601A46884201D1D86910BD10F8014B94612C
S31500000B70F7E700BF00400E4000C00140F8B504464C
S31500000B801D4616460F4600F0D7FFDDE90612204641
S31500000B9000F0D8FF0023636284F838703268C4F826
S31500000BA039207268C4F83D202B0CB26884F84530B1
S31500000BB02B0AC4F8412084F8463084F84750F8BD23
S31500000BC030B585B01D4600F12803CDE9011200932A
S31500000BD000F1240200F13803294600F0D1FF05B0E8
S31500000BE030BD00002DE9F041A2B00F4616469846EA
S31500000BF0289C054660B359B352B34BB344B30121A5
S31500000C00154800F0EBFC4022002102A802F06CFD22
S31500000C10414602A800F016FB21460AA812AC00F0D5
S31500000C2011FB40220021204602F05EFD3946204697
S31500000C3000F008FB31461AA800F004FB009402AB52
S31500000C4020222946054800F00DFB22B0BDE8F081C0
S31500000C5040F20160F9E700BF00150A0000000F40EE
S31500000C6010B5044601F026FA20460021BDE81040E2
S31500000C7001F04ABA01F052BA014601F051BA1C23FA
S31500000C8050F8042F0AB9043BFAD1002BCCBF002040
S31500000C900120704730B50568046802680368C1E939
S31500000CA00054C1E902230568046802680368C1E9C3
S31500000CB00454C1E9062330BDD1E9022330B5D1E998
S31500000CC000540560046002600360D1E90454D1E970
S31500000CD00623056004600260036030BD2DE9F04123
S31500000CE004461D460E46904600211C22181D02F0A1
S31500000CF0FBFC01232B6000F0AFFC4146074604F5E0
S31500000D008070FFF7D9FF314604F5827004F58476CA
S31500000D10FFF7D2FF29463046FFF7CEFF384600F0F0
S31500000D209FFC0D4F0D4B0E4A0E490F482365636914
S31500000D30DB010BD500F090FC294604463046FFF750
S31500000D40A9FF2046BDE8F04100F08ABC2265616536
S31500000D50A065E765EBE700BF393801003939840142
S31500000D60D02484FC1C82FED88B1C81A02DE9F04F78
S31500000D708DB0044698460F46154600F06DFC04F506
S31500000D80827607F14002114604F5867B814630469D
S31500000D900392FFF791FF29465846FFF78DFF04F5AA
S31500000DA08873184605F120010293FFF785FF484630
S31500000DB000F056FC424921654249616501254249D8
S31500000DC0A165E56500F048FC04F5847907F1200A81
S31500000DD0019039463046FFF76FFF51464846FFF708
S31500000DE06BFF039A029B11461846FFF765FF0198B1
S31500000DF000F036FC354B2365354B6365A56500F081
S31500000E002BFC04F58073019008F14001184602930B
S31500000E10FFF740FF04A94846FFF73CFF019A10463A
S31500000E2000F01EFC00F018FC394601905846FFF70A
S31500000E3043FF019A104600F013FC264A2265264A13
S31500000E4062656FF42673A2F5FE221A44A265E56573
S31500000E5000F002FC514607463046FFF72DFF3846A4
S31500000E6000F0FEFB1D4A22651D4A6265A56500F07D
S31500000E70F3FB414607464846FFF70CFF384600F0AD
S31500000E80EFFB00F0E9FB04A907463046FFF714FF25
S31500000E90384600F0E5FB134A2265134A6265A565EC
S31500000EA000F0DAFB029B044608F120011846FFF722
S31500000EB0F1FE204600F0D4FB0DB0BDE8F08F00BF78
S31500000EC08AD11C81D91C83D11C81E11CD01482CB10
S31500000ED01481E11C8CE11C811C84D91CE014D814FB
S31500000EE01482E11C84D31482D11CE0142DE9F04154
S31500000EF0044690B00F46244E0521904600F0B3FB01
S31500000F0000232360236363630FCE08AD0FC596E805
S31500000F100F0085E80F0008AA6B4607F1400120463E
S31500000F20FFF7DCFE00F098FB04F586750646694679
S31500000F3004F58270FFF7C0FE39462846FFF7BCFE6F
S31500000F4007F1200104F58870FFF7B6FE304600F081
S31500000F5087FB0E4B23650E4B63650E4BA365012382
S31500000F60E36500F079FB08F12001064604F5807080
S31500000F70FFF790FE41462846FFF78CFE304600F00C
S31500000F806FFB10B0BDE8F081A43700008AD11C8148
S31500000F90D91C83D11C81E11C2DE9F04FA5B01D465B
S31500000FA00446CDE9001205A81C22002102F09CFB94
S31500000FB04FF0010820220021284605F12007CDF830
S31500000FC0108005F1400A02F08FFB202200213846EE
S31500000FD002F08AFB20220021504602F085FB052103
S31500000FE0204600F040FB00232360FF262363636353
S31500000FF07211019806F01F0350F8222008FA03F335
S31500001000134206F1FF3102D10E460029F0D100F05D
S3150000101023FB04F582733946804618460293FFF790
S315000010204BFE404600F01CFB7A4B7B4A236562650B
S315000010307A4AA26500F010FB04F5807914A980466F
S315000010404846FFF727FE404600F00AFB00F004FB87
S31500001050294680464846FFF72FFE404600F000FB33
S315000010606F4A704B22654FF486726365A26500F085
S31500001070F3FA04F5867883460CA94046FFF70AFE84
S315000010801CA94846FFF706FE584600F0E9FA00F0AC
S31500001090E3FA029B0393514683461846FFF70CFE7C
S315000010A0584600F0DDFA604B23650123636500F0C6
S315000010B0D3FA04F5847B294602905846FFF7FCFDD7
S315000010C0029A104600F0CCFA584A226502F1D9423B
S315000010D002F5DE1202F595626265A2F5861201231B
S315000010E0A2F2BA42A265E36500F0B6FA1CA9029024
S315000010F05846FFF7E1FD0CA94046FFF7DDFD029AD1
S31500001100104600F0ADFA4A4A22654A4A62654A4AE2
S31500001110A26500F0A1FA2946029004F58870FFF74F
S31500001120B9FD029A104600F09BFA00F095FA039B6F
S31500001130029039461846FFF7BFFD58465146FFF75D
S31500001140BBFD14A94046FFF7B7FD029A104600F012
S3150000115087FA3A4B23653A4B636500F07DFA5146B0
S3150000116083464846FFF796FD39464046FFF792FD0F
S31500001170584600F075FA012106F01F0301FA03F341
S315000011807211019951F82220134217D02B687BB9AE
S315000011902846FFF774FD58B12B6A4BB93846FFF75E
S315000011A06EFD28B12B6C1BB95046FFF768FD60B980
S315000011B02B46009A29462046FFF7D8FD16F1FF3642
S315000011C0BFF425AF25B0BDE8F08F009BAC4603F118
S315000011D0200E18685968624603C208337345944660
S315000011E0F7D1BC4603F1200E18685968624603C25F
S315000011F0083373459446F7D10DF1100EBEE80F0083
S3150000120005F1400CACE80F009EE80F008CE80F00DB
S31500001210D4E700BF8AD11C81821CC00C0C0C0100D3
S31500001220C00C0C83D91C83D88AD11C83DA0C811498
S315000012308CE11CD01484E31482D11C01D81483D110
S315000012401CC00C0110B520220C46002102F04CFAFD
S3150000125004F12002013812F8013D00F8013FA242D4
S31500001260F9D110BD2DE9F04FBBB0894604460021E7
S3150000127090460AA860229A46449F02F035FA6022F8
S31500001280002122A802F030FAB9F1000F00F01E8109
S31500001290BAF1000F00F01A81002F00F01781B8F1A3
S315000012A0000F40F3138100232360236363636368A5
S315000012B0884E43F0100363600C21204600F0D3F9FA
S315000012C0636823F4406343F400636360636823F454
S315000012D0407343F4007363600FCE2AAD0FC596E8E2
S315000012E00F0085E80F0000F0B7F904F58476834611
S315000012F03946304604F58675FFF7DEFC2AA92846EE
S31500001300FFF7DAFC584600F0ABF90122724B236571
S3150000131062656269D20104D440F202603BB0BDE866
S31500001320F08F391F082251F8040F002800F0C680FC
S31500001330019300F091F907F1200B009059463046D1
S31500001340FFF7BAFC2AA92846FFF7B6FC009A104612
S3150000135000F086F9019B2365012363656369DB0160
S31500001360DAD507F11C02082352F8041F002900F001
S31500001370A980B8F1200FA8BF4FF020082022002135
S3150000138032A802F0B1F908F1FF30CC4620F0030391
S315000013903AA940330B441CF8012B00F00301C900A5
S315000013A08A4053F8601C0A4343F8602CACEB0903EF
S315000013B0434500F1FF30E9DB00F04EF932A98046E3
S315000013C03046FFF779FC404600F04AF9434B236567
S315000013D000F042F904F58078814632A94046FFF7CD
S315000013E059FC484600F03CF92AAA02AB5946204669
S315000013F0FFF774FC00F030F904F58879834602A9FA
S3150000140004F58270FFF758FC32A94846FFF754FCF2
S3150000141039462846FFF750FC584600F021F9304B74
S31500001420236503F1FA43A3F50063636500F014F93D
S3150000143032A983464846FFF72DFC02A94046FFF72E
S3150000144029FC584600F00CF90AAB32AA2549204679
S31500001450FFF7A2FD22AB02AA51462046FFF79CFDEC
S315000014600AAA11462046FFF741FD22AB19460AAAF1
S315000014702046FFF77BFC22AA11462046FFF736FDE1
S3150000148000F0EAF80C218046204600F0ECF822A98C
S315000014903046FFF711FC39462846FFF70DFC40465B
S315000014A000F0DEF8104B2365104B6365636913F09B
S315000014B0807F40F2046018BF00202FE7013A7FF4D6
S315000014C032AF29E7013B7FF44FAF25E740F20160D9
S315000014D024E700BFC43700003035DA1030D00C01E5
S315000014E030E11C84E43700003035DA143938010065
S315000014F01FB5124B1A6842F480121A60D3F8C02046
S3150000150042F00102C3F8C020FFF70AFA4FF47A232B
S31500001510B0FBF3F00A4B0D2218600021684602F07A
S31500001520E3F801238DF8003069460A2305488DF853
S31500001530023000F0DBF905B05DF804FB00400E4018
S3150000154038010020008001400C4A0D4B10B5546A4A
S315000015501B68A4B213FB00400A4B80B21880A0425D
S31500001560094B2CBF002401241C70134611B15A6A82
S315000015708242FCD101225A619A6110BD008001406D
S315000015803801002034010020360100200A4B1A7869
S315000015900A4B22B1D86810F0010003D17047DA680F
S315000015A0D20707D4586A064B1B88984234BF0020DE
S315000015B0012070470120704736010020008001405D
S315000015C034010020044BD3F84421D20703D4D3F8C6
S315000015D040211042FBD1704700400E40C0F3032269
S315000015E0013A38B50546092A13D8DFE802F0231375
S315000015F01212051619121C20104C0020C5F30435D2
S3150000160008B1FFF7DFFF04F1047405EBC404A4007E
S31500001610216038BD00200A4CF0E70120094CEDE7B7
S315000016201020094CEAE74FF48030084CE6E700202A
S31500001630074CE3E70020074CE0E700BFB0400E4050
S31500001640C0400E40E0400E40E8400E40F0400E40E4
S3150000165050410E4000400E40EFF3108072B67047C6
S3150000166000B962B670470E2910B543680DD801223D
S315000016708A4047F2E004224223F01F0306D140F6D7
S315000016801F74224201D01943416010BD41F0100180
S31500001690F9E70000F0B54AB130261E4C0125464355
S315000016A08D4034440BB304F1C064256030244443B8
S315000016B004F18044072904F5204419D865688E0092
S315000016C00F27B74025EA070502FA06F63543656097
S315000016D052B9012202FA01F1302250430D4A024466
S315000016E0A3B102F1C0621160F0BD04F18064DCE7D1
S315000016F001F18045083DA668AD000F27AF4026EAF8
S31500001700070602FA05F53543A560E1E702F18062B6
S31500001710E9E700BF0CA000400F4A70B5002308257A
S315000017208B4201D1002070BD50F8234094610B4CD0
S31500001730D5600133D669F60705D514B96FF00200F6
S31500001740F1E7013CF6E7002CF8D0D469A407E7D509
S315000017506FF00100E7E700BF00000E40809698009A
S31500001760094A0A4BD969C90705D512B96FF00200B3
S315000017707047013AF6E7002AF8D001221861DA60CC
S31500001780D86940F3800070478096980000000E40AC
S3150000179009B1FFF7C1BF084670470000234B2DE98A
S315000017A0F0470F4641F671311E6C1964996841F095
S315000017B001018146B6B299604FEA9208BA46002501
S315000017C045450ED30020D9F800203B689A420ED03A
S315000017D04846FFF7C5FF50B901213846FFF79CFF81
S315000017E005E009EB85042046FFF7BAFF48B10F4B29
S315000017F09A6822F001029A600EB100221A64BDE8CE
S31500001800F087C4F30A04C4F50064A408A8EB050332
S315000018109C4228BF1C4621465046FFF7B9FF0028C8
S31500001820D1D125440AEB840ACAE700BF00000E4066
S315000018301E4B41F671311A6C10B51964996841F066
S315000018400101996001211861D960D9694C0792B2EA
S3150000185009D5996821F0010199600AB100221A643C
S315000018604FF0FF301FE00221114CD9601946D869AC
S31500001870C00700D56CB9C8698B6810F0020023F068
S3150000188001038B6007D00AB100230B646FF00100DF
S3150000189009E0013CEBE724B902B10C646FF00200E9
S315000018A001E00AB1086410BD1046FCE700000E40D6
S315000018B080969800FFF772BF0B4A536911699B0027
S315000018C003F03C03C1F381110B438370136903F0EA
S315000018D03F0343709369D26903F0F003C2F3031226
S315000018E013430370704700BFD0FF0FE02DE9F04FA0
S315000018F00C780CB902234360002343624B78CA7804
S3150000190091F802B08D7A91F808A091F8069091F8B6
S315000019100780002B4B7A4FEA024214BF4FF0400E6D
S315000019204FF0000E42EA0B62002B14BF8023002307
S3150000193042EA0A02002DCD7A42EA892214BF4FF00C
S31500001940200C4FF0000C42EA0822002D0D7B42EAE3
S315000019500E0214BF102700271343002D0D79497975
S3150000196043EA0C0314BF082600263B43002D14BF90
S315000019704FF4005500253343002914BF4FF0805122
S3150000198000212B430B4303600CB101234360BDE8E8
S31500001990F08F00001C4AD2F8B03013B543F00403B0
S315000019A00021C2F8B030084601230422FFF772FE78
S315000019B000230093009B632B20DD002101230222DC
S315000019C00846FFF767FE00230193019BB3F5FA7FF4
S315000019D017DB0E4B00221C68114610460123FFF749
S315000019E059FE094AD2F8B03014F1FF3023F004034F
S315000019F018BF0120C2F8B03002B010BD009B013301
S31500001A00D7E7019B0133DFE700400E408003144215
S31500001A1030B50568046802680368880785B011D088
S31500001A20CDE90054CDE902236C460B4604AD2246AF
S31500001A3003CAAA4218605960144603F10803F6D196
S31500001A4005B030BDC1E90054C1E90223F8E77FB50E
S31500001A508B07024615D00B466D4601F11006186835
S31500001A6059682C4603C40833B3422546F7D1009B78
S31500001A701360019B1360029B1360039B136004B009
S31500001A8070BDD1E90054D1E90203156014601060FD
S31500001A90F4E700F10473102A30B54FEA43131AD164
S31500001AA001221A60D1E90054D1E90223C0F810518D
S31500001AB0C0F81041C0F81021C0F81031D1E9045423
S31500001AC0D1E90623C0F81051C0F81041C0F8102122
S31500001AD0C0F8103130BD00221A60D1E90054D1E9B6
S31500001AE002234562446242624362F3E7F0B58C0723
S31500001AF089B006460B4615460FD0082A6C4610D10B
S31500001B0001F1100718685968224603C20833BB4220
S31500001B101446F7D12A4669463046FFF7BAFF09B0A0
S31500001B20F0BD01F1200718685968224603C2083340
S31500001B30BB421446F7D1EDE718B12422002101F08B
S31500001B40D3BD704770B50E461546044690B189B1AF
S31500001B502422002101F0C8FD802D02D0B5F5807F3A
S31500001B600BD12046EA0840F8045B314601F0B1FD8E
S31500001B70002070BD6FF02100FBE76FF02200F8E750
S31500001B802DE9F04F814685B088469B461646F2B150
S31500001B901768B9F1000F00F0B5800F9B002B00F01D
S31500001BA0B180109B002B00F0AD80BBF1000F00F060
S31500001BB0A9800E9B002B00F0A580D9F80030802B61
S31500001BC003D0B3F5807F40F0A08000240DE01746D7
S31500001BD0DFE7A7B10F9B0E9A1B5DD25D5340109AAB
S31500001BE00137135507F00F0701344445F1D3002E92
S31500001BF000F08E803760002005B0BDE8F08F00F061
S31500001C0089F84FF44043476003600546FFF724FD1B
S31500001C10D9F80030802B824614BF1022082209F121
S31500001C2004012846FFF762FF05F18403184659466A
S31500001C300093FFF70CFF5046A8EB040A2AF00F0AA0
S31500001C40FFF70EFDA244032354451AD10F9B03EB65
S31500001C50040A109B1C440F9B434401930323019ADF
S31500001C6092452DD1FFF7F8FC594604460098FFF738
S31500001C70CFFE2046FFF7F4FC284600F055F8444610
S31500001C80B3E74822AA600522AA602A699107FCD414
S31500001C90AB600293FFF7E0FC0F9B0190191905F169
S31500001CA0A000FFF7D4FE109B05F180001919FFF77D
S31500001CB0AFFE019A1046FFF7D3FC1034029BC3E730
S31500001CC0AFB94822AA600522AA602A699207FCD405
S31500001CD0AB600393FFF7C0FC0E99029005F18000FC
S31500001CE0FFF796FE029A1046FFF7BAFC039B0E9981
S31500001CF01AF8012BC95D01374A4004F8012B07F099
S31500001D000F07ACE76FF0210076E76FF0220073E76C
S31500001D10304671E7024B034801221A60704700BF44
S31500001D200416C84300000F40054B984206D103F144
S31500001D306E7303F58B33043300221A60704700BFBD
S31500001D4000000F402DE9F04F99B007460E46904629
S31500001D501D46FFF7DFFF04462FB1022F00F2E58094
S31500001D600423036000E0076000236360E3646268A5
S31500001D7022F4406262602363636356F8232012BA3A
S31500001D804DF823200133082BF7D1FFF765FC009BA4
S31500001D90C4F80431019BC4F80431029BC4F8043131
S31500001DA0039BC4F80431049BC4F80431059BC4F8B2
S31500001DB00431069BC4F80431079BC4F80431FFF7CD
S31500001DC04FFCDFF874A15A4B2365002608F003097F
S31500001DD0229B9E4239D1AB0700F08A80FFF73CFC7C
S31500001DE0D4F80061D4F80011D4F80021D4F80031F9
S31500001DF0CDE90061CDE90223D4F80061D4F80011E1
S31500001E00D4F80021D4F80031CDE90461CDE90623E8
S31500001E102E46FFF725FC08AF6B461A4603CABA42A0
S31500001E2030607160134606F10806F6D12046FFF7CA
S31500001E307BFF2B1F1C3553F8042F12BAAB421A60D6
S31500001E40F9D1002019B0BDE8F08F08EB861BB9F177
S31500001E50000F0FD008AA0BF1400CDBF80000DBF8EE
S31500001E600410134603C30BF1080BE3451A46F4D1DD
S31500001E700DF1200BFFF7F0FBDBE90131DBF80C205D
S31500001E80DBF80070C4F8A471C4F8A431C4F8A41136
S31500001E90C4F8A421DBE90531DBF81C20DBF810705F
S31500001EA0C4F8A471C4F8A431C4F8A411C4F8A421D8
S31500001EB0DBE90931DBF82C20DBF82070C4F8A471CB
S31500001EC0C4F8A431C4F8A411C4F8A421DBE90CC1F8
S31500001ED0DBE90E23C4F8A4C1C4F8A411C4F8A421F4
S31500001EE0C4F8A431FFF7BCFB0136C4F850A06FE775
S31500001EF0FFF7B2FBD4F80061D4F80011D4F8002142
S31500001F00D4F80031C5E90061C5E90223D4F80061BF
S31500001F10D4F80011D4F80021D4F80031C5E90461E1
S31500001F20C5E90623FFF79CFB80E702488AE700BF66
S31500001F30888AC80180AFFFFF070D81012DE9F347AD
S31500001F400228144680460E461F46DDE90A924ED800
S31500001F501CB9002002B0BDE8F08713683F2B42D8B9
S31500001F60516809B1002F3ED1B8F1010F3DD0224D85
S31500001F702249B8F1020F18BF0D4603F03F00E318DF
S31500001F80136022BF53680133536090B3C0F1400A17
S31500001F90544522D331465246484401F09AFB012368
S31500001FA000934A463B4629464046A4EB0A04FFF7FF
S31500001FB0C9FE3F2C56440DD93D46A309009332462F
S31500001FC03B4629464046FFF7BDFE24F03F031E442C
S31500001FD004F03F04002CBCD0002022463146484481
S31500001FE001F077FBB5E73D46C7E7054DC5E7054870
S31500001FF0B0E73F2CF1D9E0E7643800002438000050
S315000020004438000080AFFFFF2DE9F041012886B07B
S3150000201004460E4690461D4604D045D3022841D0BC
S3150000202022483CE01C272A68D3008DF80F3053095C
S315000020308DF80E30530B8DF80D30530D8DF80C3096
S315000020406B68D90001EB52718DF80B1002F03F025C
S315000020505909372A8DF80A104FEA53314FEA53537C
S3150000206094BFC2F13802C2F178028DF809108DF8DA
S3150000207008300F493346CDE900852046FFF75EFF5D
S3150000208008220DEB02013346CDE900852046FFF715
S3150000209055FF3A4631460C9801F01BFB002006B06E
S315000020A0BDE8F0812027BEE71427BCE780AFFFFF1D
S315000020B08438000018B16C22002101F015BB70476E
S315000020C007B590F868300190002B00F128030093C3
S315000020D000F1080314BF01200220FFF72FFF03B011
S315000020E05DF804FB07B590F868200091002A0346C6
S315000020F000F1280200F1080114BF01200220FFF7B9
S3150000210083FF03B05DF804FB00239942D4BF00218E
S315000021100121C0E9003380F868107047FFF7D0BF8F
S31500002120FFF7E0BF0020704700207047002070478F
S315000021300020704740F628031B681869704728235B
S315000021401868704740F62803186870472823044A21
S315000021501B68196891420CBF18690020704700BFC0
S31500002160AD1007B001207047004870474A43E00FA2
S31500002170004870476A43E00F004870478642E00F08
S3150000218038B501213448354CFFF728FA0121344887
S31500002190FFF724FA01214FF48A40FFF71FFA0121C5
S315000021A03048FFF71BFA40F6AA630025E3602E4A83
S315000021B0256041F2050365666360A5606561E564B7
S315000021C0A2646567A567E567636023682360FEF719
S315000021D0A7FB00F5E1404FF4E1134001B0FBF3F03B
S315000021E0224B203803EAC00001236061042218460E
S315000021F00E21FFF74FFA01231A460F211846FFF763
S3150000220049FA40F60913A367032205236267E360D0
S31500002210174B4FF0E06119604FF440211D62DD62FB
S315000022205D63DD66C3F880101249C3F88850C3F8B1
S315000022308450C3F898101049C3F8B0100F49C3F87A
S31500002240B850C3F8B4500A600122DA6303F1C063E0
S31500002250083302221A6038BD4041050000000140E3
S3150000226000250A0000220400F9FF0100F8FF7F00A4
S3150000227000200E40C438000001000C0028200E4447
S31500002280084B986A10F0020005D0074A0223136033
S315000022909360012070471B6A9B07FBD4034B022205
S315000022A01A60F6E700200E4020200E4428200E4437
S315000022B07F2938B50546144624D8FFF7E1FFA8B9AB
S315000022C041F2062038BDE85C985401338B42FAD1BE
S315000022D00E490888013B63F30E100D4B088002225D
S315000022E0C3F8C810DA6324B90020EBE70023094AD3
S315000022F0ECE7FFF7C5FF0028FBD0074A13699B06EA
S31500002300FCD5F1E741F20310DCE700BF0001002035
S3150000231000200E40400300200000014008B50146A1
S31500002320FFF7AEFF0028FBD0054B1A46186940069A
S31500002330FCD5596313699B06FCD5002008BD00BF78
S31500002340000001400E4BD3F8940040F2011398426E
S315000023500FD040F2022398420DD00A4BC01A0A4B06
S315000023601B6883420AD02ABFC3F50073C01AC0187F
S3150000237070470020F3E74FF48070F0E700207047C5
S3150000238000200E403C0100203C0300202DE9F843CC
S31500002390089F04460D461646FBB9FFF7D3FF2149B1
S315000023A0DFF888E00B68204FA84228BF284622465F
S315000023B004EB000C4FF0010800244FF002096245BF
S315000023C01DD104B10B6006B1306041F20423A8426E
S315000023D034BF18460020BDE8F8832FB1FFF788F810
S315000023E000213846FFF7B0F8FFF7ACFFA842D4D279
S315000023F0002FF9D0FFF7CAF80028F5D0CDE71EF870
S31500002400034002F8014B0133B3F5007F04D1C7F84E
S31500002410009000230124D2E7B3F5807F08BFC7F8F8
S315000024200080F7E73C03002008200E463C01002010
S3150000243007B50123009100221946FFF7A7FF03B055
S315000024405DF804FB10B10A4B02221A6071B1084A0A
S315000024500849012313609360074AC2F89810074998
S3150000246000200860D363064B02221A6000207047E2
S3150000247020200E44C438000000200E403C030020FB
S3150000248008200E4607B54FF47A710DF10700FFF7E5
S31500002490CFFF50B99DF80730313BDBB2022B01D894
S315000024A0034AD05C03B05DF804FB0120FAE700BFE5
S315000024B004390000FFF764BE10B540F6280392B059
S315000024C01B6813499C684522684601F002F9C4F36B
S315000024D00363092B8CBF373330338DF81430C4F3C4
S315000024E00343092B04F00F048CBF37333033092C18
S315000024F08CBF373430340122452168468DF81630BA
S315000025008DF81840FFF7D4FE002012B010BD00BFB2
S315000025101A3900002DE9F047F8B000248DF80F4075
S31500002520FEF7E6FFB64EDFF8F082DFF8F0923C27C2
S315000025300125062DFDD8DFE815F009000D00120073
S31500002540330053004C01C1000425F2E7FFF7B4FF46
S315000025500125EEE7FFF796FF3C270546E9E701224E
S315000025601121A848FFF7A4FE202317AA05A954A8FD
S3150000257000F0D6FC28220021A14801F0B5F8FF237F
S31500002580012105207370FEF7DFFFFFF7DBFE18B1B0
S3150000259001210020FFF756FF00F04EF90325C8E79A
S315000025A04320FFF7BBFE00214FF47A70FEF7CCFF05
S315000025B0FFF7C8FE18B9FEF7E9FF0028F8D0FFF7C5
S315000025C0C1FE0028C0D1013FB3D11820FFF7A6FEF7
S315000025D01820FFF7A3FE1820FFF7A0FE0025A8E7A6
S315000025E0002185220DF1C90001F07EF8002140F698
S315000025F0B830FEF7A9FFFFF7A5FE78B34FF47A735C
S3150000260000930123194604AA0DF1C900FFF7BEFE87
S315000026109DF8C930012B0DD140F6B83200928421C5
S3150000262004AA0DF1CA00FFF7B1FE049B842B0446F1
S3150000263018D1C8B90DF10F010DF1C90000F006F966
S3150000264040F607139842044614D1B3780BB1F378D9
S3150000265013B918238DF80F3006251DE0FEF796FFF7
S315000026600028C8D040F2047415208DF80F00FFF73B
S3150000267055FE5EE780B99DF8C930012B0CD1624B3F
S31500002680009333AA8023314654A800F083FC044605
S3150000269010B118238DF80F309DF80FA0BAF1180F5E
S315000026A0504608BF0625FFF739FEBAF1180F7FF42A
S315000026B040AF5046FFF732FE5046D8E701210020D2
S315000026C0FFF7C0FE01210A20FEF73EFF9DF80F30FE
S315000026D0062B4FF0010208D140F607139C4204D1A5
S315000026E04A481B21FFF7E4FD78E71A214846FFF721
S315000026F0DFFDA4F51063B3F5E06F39BF1821444838
S31500002700444810210122FFF7D3FD41F201039C4208
S3150000271049D02FDC40F603139C4246D01FDC40F61E
S3150000272001139C4247D040F602139C4245D09DF8C7
S315000027300F00000909288CBF37303030FFF7EEFD57
S315000027409DF80F0000F00F0009288CBF373030309D
S31500002750FFF7E4FD0D20FFF7E1FD0A203CE740F618
S3150000276005139C422BD024DB40F606139C42DED197
S3150000277027231BE041F207039C4214D00ADC41F2F6
S3150000278005039C421FD022DC41F204039C42CED1B9
S3150000279050230BE041F209039C4212D015DB41F2B3
S315000027A00A039C42C3D14F2300E021238DF80F304A
S315000027B0BDE72223FAE72323F8E72423F6E72523B8
S315000027C0F4E74123F2E74323F0E74423EEE745230A
S315000027D0ECE7B3784BB3F3783BB333789B071FD55D
S315000027E040F6280372681B689B689A4204D9FFF773
S315000027F0ADFC716A00F092F901221321404671E79F
S31500002800C0030020B5390000703900009A39000075
S31500002810C63900005F390000073900008039000022
S3150000282040F2012000F0CEF9E6E740F2032000F086
S31500002830C9F9D3E670470000024A00231370024A22
S3150000284013707047E8030020E903002038B50378C9
S31500002850042B05460C4650D008D8012B0AD0032B72
S3150000286050D11823237040F608100DE0182BF8D02D
S31500002870432BF5E7264B42781978D9B9012A04D0BB
S315000028801523237040F6041038BD1A70AB781A442D
S31500002890FF2AF5D100228021E81CFEF746F995F8BB
S315000028A08320C0F30F239A4216D01523237040F6D7
S315000028B00210E9E7174B1B78934204D106232370D5
S315000028C040F60610E0E70133DBB29342DED0152373
S315000028D0237040F60510D7E795F88430C0B28342DE
S315000028E004D01523237040F60110CDE7094B6A7812
S315000028F01A70062323700020C6E706230B7040F6E5
S315000029000710C1E71823237040F60310BCE700BF89
S31500002910E9030020E8030020F0B50F4B85B06C46B4
S31500002920024603F11007264618685968254603C56E
S315000029300833BB422C46F7D104AB501E13F8011DD9
S3150000294010F8012F914204D1B342F7D1012005B00E
S31500002950F0BD0020FBE700BFDE390000C0F30A032C
S315000029602DE9F04105460F4616460BB900F076F9FB
S3150000297005F5006424F4FF6424F0070405EB06085B
S31500002980A04506D8324639462846BDE8F04100F053
S315000029906CB9204600F062F904F50064F0E770B502
S315000029A09EB0446B0546FFF7CDFB06462046FFF773
S315000029B0B3FF48B3237C012B28D86369012B25D1AB
S315000029C0A4693369A34221D8A5421FD8B4F5802F44
S315000029D01CD803A8FEF744F9621B294603A8FEF794
S315000029E049F903A8FEF748F9FFF7BEFB0546FFF7CE
S315000029F0BFFB2B46009004F12002214603A8FEF7F8
S31500002A00F1F8B0FA80F040091EB070BD0020FBE777
S31500002A1070B504460E461546FFF794FB0369A342BC
S31500002A200AD8426963199A4206D32A463146204695
S31500002A30BDE87040FFF792BF70BD00002DE9F04180
S31500002A40154607468846FFF77AFB104B02689A42FE
S31500002A5019D1FFF777FB0646FFF778FBC419631910
S31500002A60B3F5802F0FD83FB9FFF770FB7369834228
S31500002A7002D9306900F0F2F82A4641462046BDE800
S31500002A80F041FFF76BBFBDE8F08100BFAD1007B0A6
S31500002A90F8B5D0E9006706F160460446456BFFF7D6
S31500002AA051FBB6F5F84F01D90020F8BD0369BB42CA
S31500002AB0FAD8B7F5802FF7D84033AB4202D8B5F530
S31500002AC0802F05D9FEF720F880F00100C0B2ECE7B0
S31500002AD0FEF71AF820B12046BDE8F840FFF75FBFC1
S31500002AE02846FFF719FFA8B12B7C012BDCD86B69B0
S31500002AF0002BDAD0022BEED1AB69C4F104011944E4
S31500002B004FF0FF322046FEF71DF8034BC31A58421A
S31500002B105841CAE70120C8E7E320BBDE08B54FF0FD
S31500002B20FF32FEF70FF8044B984203D140F209201A
S31500002B3000F048F8002008BDE320BBDEB1F5BE7FFB
S31500002B4010B5044610D34FF4BE72002100F0CCFD40
S31500002B500023637004F5807204F1B80104F12800C3
S31500002B60BDE8104000F0DCB940F2052010BD13B5F9
S31500002B70044600910146283000F00CFAC4F87801AA
S31500002B8018B141F20703984209D1A3784BB1E27814
S31500002B9040F2032040F20223002A08BF184602B082
S31500002BA010BD40F20120FAE74FF000534FF20F023A
S31500002BB018805A8070474FF000534CF23C325A80CE
S31500002BC0704700004FF000534FF20F025A800A4A36
S31500002BD01880136823F4E06343F400731360BFF3B3
S31500002BE04F8F0649064BCA6802F4E0621343CB6076
S31500002BF0BFF34F8F00BFFDE700500E4000ED00E031
S31500002C000400FA054FF000534FF20F015A888A422A
S31500002C1001D1188870473AB91B88012B40F202206F
S31500002C2018BF4FF4007070474FF40070704707B537
S31500002C3003469B0753BF6FEA01414FF6FF7343EA12
S31500002C4001416FEA11410422019120F003000DEBCE
S31500002C500201FEF72FFE03B05DF804FB08B5FEF790
S31500002C60E7FDB0FA80F0400908BDF8B540EA020376
S31500002C701446DA0705460E4601D50020F8BD0CB904
S31500002C800120FBE7830721D50988FFF7D0FF00283D
S31500002C90F3D1023C032C05F1020506F102060BD91D
S31500002CA024F003073A4631462846FEF703FE00287D
S31500002CB0E3D13E443D44E41B002CE1D03188284654
S31500002CC0FFF7B5FFB0FA80F04009D7E7032CE7D845
S31500002CD0F4E770B5D1E90152AA4205D290F8403026
S31500002CE02B449B1A402B10D9002012E00A6890F85A
S31500002CF04040D65C90F84120224402F03F02013366
S31500002D00013486548B6080F840408B689D42EDD834
S31500002D10012070BD2DE9F8431746D1E90125521B64
S31500002D2090F840509DF820909DF824802A449342C4
S31500002D3004460E4657D9FFF7CCFF00285DD1122373
S31500002D4084F8463041F20200BDE8F88394F8412049
S31500002D50A25C7A5594F84120013202F03F0284F8D1
S31500002D60412094F84020013A84F84020013594F837
S31500002D70402012B1AB42E9D11D46D6E901128A4282
S31500002D8001D2AB4231D8AB42D9D1D4F888202946FA
S31500002D903846FDF7D7FEC4F88800B9F1000F04D015
S31500002DA02A463946E06CFDF765FFB8F1000F08D0FA
S31500002DB094F843302BB12B463A463946A06CFDF7C2
S31500002DC0FFFE94F8433043B1E36DA26D2B4493426A
S31500002DD0E36524BF002384F84330636D1D446565B5
S31500002DE041F20300B0E70025C1E731688A5C7A55F5
S31500002DF0B2680132B2600135BFE70020A4E70000E7
S31500002E007FB50023CDE90033082315460DEB0302F9
S31500002E100446FFF77FFF41F203039842064626D198
S31500002E2094F8433063B108220DEB0201E06CFDF724
S31500002E3021FF08230DEB03021146A06CFDF7C0FE2F
S31500002E40039A6A6094F84320029B2B605AB9094A98
S31500002E50934208D0084A934205D008220DEB02019E
S31500002E60E06CFDF707FF6B6823650023636530465A
S31500002E7004B070BDF70A0AF7FC0404FC2DE9F84318
S31500002E80044658680D4616461F46002843D08B0751
S31500002E9043D1FFF74FF9216E00F1040C06EB01094F
S31500002EA0CC451DD800F11C02914219D28C456346CF
S31500002EB038BF0B46591AA3EB0C00914594BFC3EBE0
S31500002EC00909C3EB020905EB010868304A46414689
S31500002ED0204400F0FEFB4A46FF21404600F004FC79
S31500002EE0FFF734F9226E031D93420AD3B118083056
S31500002EF0814206D39B1AEA58C4F880204FF0FF326D
S31500002F00EA50D7E900383246206E2946C047236E7C
S31500002F101E4426660020BDE8F88341F20200FAE767
S31500002F20F8B504464FF0FF36154603F0200300229D
S31500002F3080F84620A0F8402080F8432080F84520FD
S31500002F4080F84420C0E918220F4680F84230C0F8C5
S31500002F5088601822FF21683000F0C6FBC4F8806044
S31500002F60C4F88460C4E91275FFF7E2F818B117B91E
S31500002F7041F20B00F8BDFFF7D9F830B1002DF7D0BC
S31500002F80E06CFDF76DFE0020F4E7002DF8D1284631
S31500002F90F0E700002DE9F04F9BB0CDE9072303933E
S31500002FA0249EDFF800B40023044689460993984618
S31500002FB0099A039B9A4257D294F84630122BF8D8B6
S31500002FC0DFE813F05B00700054009A00B8013B0084
S31500002FD03200D5013B00CF013B00CF01B4025203C2
S31500002FE013001D032103490252030027636D0F2BB3
S31500002FF041D801251023019700950AAA07A9204662
S31500003000FFF788FE41F2030398427AD1D4F848A02C
S31500003010FFF7B2F88023CDE900030BAA2B46022165
S315000030205046FDF7ABFDE1E70125D4E914329A429B
S31500003030C0F01B8184F84650BAE70DF1280AD4E99E
S315000030401452AA42099916D2089BAD1A94F8402048
S315000030505B1A032D134440F2A781032B00F2CB81A8
S3150000306007A92046FFF735FE00204AE00025636DDC
S31500003070072B40F2C380012311E005AA07A92046C9
S31500003080FFF7BEFE41F2030398423AD1069B236541
S3150000309000236365059AB84B9A422DD1022384F822
S315000030A0463085E705AA07A92046FFF7A9FE41F2A3
S315000030B00303984225D194F84420059B22B1AF4AD8
S315000030C0934219D10C23EAE794F84220D1074FD551
S315000030D094F84320002A40F0CA82A94A934241D07C
S315000030E017D8A84A934207D00ED8A34A934203D0D2
S315000030F002F1B642934215D1122384F8463041F2CA
S3150000310001001BB0BDE8F08F9F4A9342F4D09F4A5E
S31500003110F0E79F4A93421BD00CD85B4543D09D4AAB
S31500003120934217D0122384F8463005A8FEF7FAFF1B
S31500003130D8B1E4E7984A9342DED0984A9342DBD06E
S315000031408E4A9342EED1FEF7F1FF0028BAD0D3E7BC
S315000031500E23A4E70F2384F84630236DA3650023CE
S31500003160E36525E7122384F8463041F20800C8E7F4
S315000031705B4514D000F27F82834A934207D0834A8C
S31500003180934206D07F4A93420FD1062387E7042352
S3150000319085E7072383E7092381E70B237FE794F875
S315000031A04330002BA8D1102379E705A8FEF7BAFF14
S315000031B0D0B11123059884F84630C4F88C00FEF788
S315000031C0B3FF94F842309A0680467FF5F1AE0028A8
S315000031D03FF4EEAE4368002B3FF4EAAE2046984734
S315000031E000283FF4E5AE8AE7122384F8463094F8C7
S315000031F04330002BB9D041F2040082E7012300934B
S31500003200019508230AAA07A92046FFF783FD41F284
S31500003210030398427FF475AF0A9B03F07F43B3F133
S31500003220407F05D0122384F8463041F2090068E752
S315000032300B9B0493DB070ED594F8423043F0010351
S3150000324084F84230FEF772FF00283FF410AF049B6B
S31500003250DF0504D50BE7FEF76BFF0028F2D012233B
S3150000326084F8463041F20A004BE7CDE900550AAA38
S3150000327007A92046FFF74EFD41F2030398427FF46B
S3150000328040AF09F1080C0AAF63460DF1400E3A460D
S3150000329003CA724518605960174603F10803F6D150
S315000032A01068186099F8003043F0010389F800307F
S315000032B06046FEF757FF00287FF4B7AE122384F866
S315000032C0463041F20C001CE70123CDE900330AAA7F
S315000032D0082307A92046FFF71DFD41F20303984284
S315000032E07FF40FAF99F8003043F0020389F80030FD
S315000032F00A9BC9F80430236D083BC9F824300B9BA0
S315000033000493FEF71CFF264A036893427FF4F7AE48
S31500003310FEF715FF049BC2689A427FF4EDAE0523C3
S3150000332084F8463094F8453043F0010384F845307C
S3150000333000236366636D072BC6D939E60423CDE9FE
S3150000334000550AAA07A92046FFF7E4FC41F2030349
S3150000335098427FF4D6AE226D0A9B0493042A01D9C3
S3150000336023660125636D032BE8D90A2397E600231C
S315000033706366082393E600BFEB17A603FC0404FC70
S31500003380F70909F7F40A0AF4F50909F5F60808F643
S31500003390FA0606FAF90707F9FD0303FDFE0101FE29
S315000033A0AD1007B0F70A0AF79D423FF659AE9D42A7
S315000033B028BF1D46032D88BF25F003050123CDE94F
S315000033C0003352462B4607A92046FFF7A3FC41F2DD
S315000033D0030398427FF495AE94F84630082B13D138
S315000033E0B7688FB13368606E2A465146B847636E38
S315000033F01D44656623E6402D28BF4025D7E74FF0DC
S31500003400FF320AF805200135032DF8D90A2B06D11B
S3150000341033462A4651462046FFF730FD0FE6052B78
S315000034207FF40DAE99F8013098077FF508AEF36882
S31500003430002B3FF404AE626E042A0AD85319062BF9
S3150000344007D90BAB9B1A1A68C4F884204FF0FF32D9
S315000034501A60F768C6E794F84230990607D5D4F89B
S315000034608C00FEF761FE804600283FF448AE012737
S315000034703FE0002B58D0B8F1000F55D0D8F81030E7
S31500003480002B51D020469847DDE90853ED1A94F8F1
S3150000349040302B4498423FF6E3ADD4E91452AD1ABE
S315000034A0402D28BF40259D4228BF1D462B46CDE90D
S315000034B000770AAA07A92046FFF72CFC41F203036E
S315000034C098427FF41EAE94F842309A0611D5B8F1B0
S315000034D0000F3FF414AED8F808A0BAF1000F3FF47D
S315000034E00EAE33462A460AA92046D04700287FF466
S315000034F008AED4E9142194F84230914203F0200337
S31500003500B7D3002B3FF4B7ADB8F1000F3FF4B3AD1E
S31500003510D8F80C30002B3FF4AEAD31462046984724
S3150000352000283FF4A8ADECE50120ADE70023CDE986
S3150000353000330AAA042307A92046FFF7EBFB41F252
S31500003540030398427FF4DDADD4F88820554B9A42A8
S3150000355005D0122384F8463041F20500D1E5FEF786
S31500003560E5FD10B9012389F8033099F80330002BE3
S315000035703ED094F845309B0707D0F5682DB104225C
S31500003580336804F184011046A847236E83B3736839
S3150000359073B31AAF4FF0FF3347F8583D04F1800874
S315000035A004224146384600F085F840B1FEF7CEFDCC
S315000035B028B10422D6E9003541461044A84704F153
S315000035C0680504222946384600F074F880B1776809
S315000035D0FEF7B0FD3368142204F16C010830B847D9
S315000035E07768FEF7A7FD0422336829461044B847DA
S315000035F0012389F802300D2384F8463034E501238F
S3150000360084F843304BE594F84450002D7FF433ADF5
S315000036104023CDE900550AAA07A92046FFF77AFB01
S3150000362041F2030398427FF46CADE06CFDF724FB96
S31500003630E76CFEF799FD8246FEF79AFD5346009029
S3150000364012AA0AA93846FDF7CDFA38B1122389F82D
S31500003650035041F2060084F8463052E5012389F80A
S31500003660033084F8443006E541F2070049E55B453E
S315000036707FF480AD40E50C4A93423FF48EAD0B4A91
S3150000368093423FF488AD0A4A93427FF48EADFEF72B
S315000036904DFD00287FF430AD94F84330002B3FF405
S315000036A011AD29E5E320BBDEFD0303FDFE0101FEAE
S315000036B0FC0404FC30B50024A24201D1002007E03E
S315000036C0035D01340D1915F8015CAB42F4D0581BAB
S315000036D030BD10B5431E0A44914200D110BD11F809
S315000036E0014B03F8014FF7E702440346934200D12A
S315000036F0704703F8011BF9E7F8B500BFF8BC08BC32
S315000037009E467047F8B500BFF8BC08BC9E46704799
S315000037100400000700000D1013001A202630384060
S315000037204800000007B0CD5E0100000003000A015A
S31500003730103200000040000000000400F0001000FD
S31500003740190900001D090000912A00003D2B000008
S315000037506F2B00000000000013B779FAC925DDB70A
S31500003760ADF3CFE0F1B614B801010000020000008D
S315000037700C3A00004000000003000A0100000000AF
S315000037800000000000000000000000000000000033
S315000037900000000000000000200000000001000002
S315000037A0050C0000FFFFFFFFFFFFFFFFFFFFFFFF0E
S315000037B00000000000000000000000000100000002
S315000037C0FFFFFFFF512563FCC2CAB9F3849E17A70A
S315000037D0ADFAE6BCFFFFFFFFFFFFFFFF00000000A2
S315000037E0FFFFFFFF96C298D84539A1F4A033EB2D11
S315000037F0817D0377F240A463E5E6BCF847422CE1FD
S31500003800F2D1176BF551BF376840B6CBCE5E316B40
S315000038105733CE2B169E0F7C4AEBE78E9B7F1AFE04
S31500003820E242E34F67452301EFCDAB8998BADCFE50
S3150000383010325476C3D2E1F0000000000000000010
S3150000384000000000C1059ED8367CD5073070DD1714
S31500003850F70E5939FFC00B316858151164F98FA757
S31500003860BEFA4FA46A09E667BB67AE853C6EF37283
S31500003870A54FF53A510E527F9B05688C1F83D9AB35
S315000038805BE0CD1980000000000000000000000091
S315000038900000000000000000000000000000000022
S315000038A00000000000000000000000000000000012
S315000038B00000000000000000000000000000000002
S315000038C000000000F00F10031C0001403C01002026
S315000038D013000000090000000001000002020000C1
S315000038E013000000F00F10031C0001403C020020F2
S315000038F013000000090000000002000001010000A2
S31500003900D3FFFFFF0205000D0A4661696C6564205E
S31500003910746F20626F6F740D0A000D0A4765636B42
S315000039206F20426F6F746C6F616465722076582EDB
S31500003930592E410D0A312E2075706C6F6164206717
S31500003940626C0D0A322E2072756E0D0A332E2065BA
S31500003950626C20696E666F0D0A424C203E20000D97
S315000039600A66696C65206572726F72203078000095
S3150000397000000000112A0000000000003D2A00009F
S315000039800D0A53657269616C2075706C6F616420F5
S3150000399061626F727465640D0A000D0A536572697F
S315000039A0616C2075706C6F616420636F6D706C65FF
S315000039B074650D0A000D0A626567696E2075706C84
S315000039C06F61640D0A000D0A584D6F64656D2062C3
S315000039D06C6F636B206572726F7220307800B8145A
S315000039E0B6F1E0CFF3ADB7DD25C9FA79B71300001C
S315000039F000000000F07F103040030020340001403A
S31500003A000000000065080000410800005928BE3388
S503037B7E
S70500000000FA
